:0400000002002132A7
:01000B0032C2
:0100130032BA
:03001B000200A43C
:20007A00751910751AFA751B00751C00751000751101751202751300751400751500751663
:0A009A000075170C75180002001E17
:03001E000202F3E8
:2000A400C0E0C0F0C082C083C0D075D008D51912751910151AE51A60030202E8751AFA02E4
:2000C40002E8AE19530E077F00BE0405BF000280030201607590FF43B03F051B7406B51B76
:2000E40003751B00AF1B8FF005F07401800225E0D5F0FBF452B0E51B2411F9E79003059339
:20010400FFE510600302015B7483251A40497404B518107403B51B0280057405B51B047F78
:20012400FF8034E51870097404B51B047FFF80277401B518097402B51B047FFF80197402FF
:20014400B518097401B51B047FFF800B7403B51806E51B70027FFF8F900202E8E5107003C6
:200164000201F27401B51A0280030201F27401B5190280030201F27F00EF240FFDE4340352
:20018400FE8D828E83E4932411F9870C0CA70CEF90031393FBC39C40030202E88D828E8375
:2001A400E493FD2411F87600BF0337E51704FE8E1724E85003751700E51724EC500C7511AF
:2001C40002E517FE24ECF5128018E51724F6500C751101E517FE24F6F512800675110085CB
:2001E40017120FBF0400500302017D0202E87408B5190280030202E820B7030202B9E510FA
:2002040060030202B4E51C70030202B47406251C50030202B47404B5180C751910751AFA55
:200224007510010202B4E5187013E51504FF8F1524F640030202B47515000202B47401B5DA
:200244001812E51304FF8F1324FA40030202B4751300805C7402B5182AE51204FF8F12242A
:20026400F650037512007402B51109E51224FC5003751100E51175F00AA4FFE512FE2FF554
:2002840017802D7403B51828E51104FF8F1124FD50037511007402B51109E51224FC5003E8
:2002A400751203E51175F00AA4FFE512FE2FF517751C00802F051C7406251C502774FAB5C2
:2002C4001C1FE510600E751800751600751400751000800DE51804FF8F1824FB5003751823
:1D02E40000751CFBD0D0D083D082D0F0D0E032758920758D0675A88843884080FE36
:1203050088BDC4A4B1A282BC80A005030402090509055E
:06005000E478FFF6D8FD84
:20002E007900E94400601B7A00900317780175A000E493F2A308B8000205A0D9F4DAF2755E
:02004E00A0FF11
:200056007800E84400600A790175A000E4F309D8FC7800E84400600C7900900001E4F0A3A8
:04007600D8FCD9FADF
:0D00210075811C120301E582600302001EC0
:0403010075820022DF
:00000001FF
